:020000040800F2
:10000000201D0020A90100081D150008410C000852
:1000100000000000000000000000000000000000E0
:100020000000000000000000000000006D1C00083F
:1000300000000000000000001F1500086D1D0008F2
:10004000BB010008BB010008BB010008BB010008A0
:10005000BB010008BB010008BB010008BB01000890
:1000600000000000BB010008BB010008BB01000844
:10007000BB010008BB010008BB0100080000000034
:10008000BB010008BB01000800000000711E000851
:10009000A51E00082D1F0008511F0008BB01000805
:1000A000BB010008BB010008BB010008A51F000838
:1000B00035200008000000000000000000000000E3
:1000C000BB01000800000000BB01000800F002F8BE
:1000D00000F03EF80CA030C8083824182D18671E10
:1000E000A246AB4654465D46AC4201D100F030F822
:1000F0007E460F3EB6460FCC0126334200D0FB1A97
:100100003343A246AB461847644B0000844B0000C3
:10011000103A02D378C878C1FAD8520701D330C850
:1001200030C101D504680C60704700000023002432
:1001300000250026103A01D378C1FBD8520700D31E
:1001400030C100D50B6070471FB51FBD10B510BD85
:1001500000F090FB1146FFF7F7FF02F085FD00F07D
:10016000A8FB03B4FFF7F2FF03BC00F007FC00009C
:1001700070B505460C46164602E00FCC0FC5103E82
:10018000102EFAD2082E02D303CC03C5083E042E4B
:1001900007D301CC01C5361F03E021782970641C08
:1001A0006D1C761EF9D270BD07488047074800478E
:1001B000FEE7FEE7FEE7FEE7FEE7FEE70448054947
:1001C000054A064B70470000811D0008CD0000085D
:1001D00020150020201D00202019002020190020BB
:1001E000F8B5042A2CD3830712D00B78491C03706E
:1001F000401C521E83070BD00B78491C0370401C17
:10020000521E830704D00B78491C0370401C521EF9
:100210008B079B0F05D0C91ADF002023DE1B08C9FE
:100220000AE0FFF7A5FFF8BD1D4608C9FD401C46C2
:10023000B4402C4310C0121F042AF5D2F308C91A87
:10024000521EF0D40B78491C0370401C521EEAD495
:100250000B78491C0370401C012AE4D40978017012
:10026000F8BD7047704770470246C80FC00781430A
:100270004B0030B54B405B009B0D20D01923DB06B3
:10028000C91801231B05994220DB0324A407042578
:100290001346AB400BD3002B04D1EB0613409B005D
:1002A000E34204D401246407002312195941FF23B7
:1002B0001B0599420BD2C9000143500F09E0CB0244
:1002C00004D501430803024305D0054830BDFF2192
:1002D000C905084330BD084607210905884330BDDC
:1002E0000000C07FF0B58B4C0F09254689B0BD4397
:1002F0007BD01D092646AE43FAD00E465E4027400D
:10030000F60F3E43254071D024012142FBD0FF244B
:10031000AD19A4042D1B039501252D05DB02DB0A75
:10032000C9022B43C90A29431E010901040F130FF7
:10033000050121431701880B820391432D098C4647
:10034000A90B1E438A039543B30B9A0396433F09B7
:10035000BA0B9403A74302962E467E430497B646F3
:100360004E19D7190C460196544305977E43371B07
:100370007646BF1B3601B646BE0B3619009676464A
:10038000BC043719009C01D3641C00946400002F46
:1003900001D001263443029E049F754366467E4386
:1003A0000496760034196E0034190094029C019E64
:1003B0001C196643751BAE46069465464519059C97
:1003C00005956C43594375460891691A0191049E3D
:1003D00001465143A41B0491611A009C0791E10658
:1003E00005D061090122114302E072E06EE061096B
:1003F000089D00272C0A2D066918049D7C412A0AB5
:100400002D066918019D6241AC0DAD026D18544175
:10041000079A910D920255196141029A6446584318
:100420005443069B059A5A43121A131B9A0E9B01BA
:100430005B187A41010B0005C3185141220A2006BE
:1004400044195A419A4200D2491C0120400281427B
:1004500003D315230226F64302E014230326F643B2
:100460002020C51AA9401746AF40DA400A4320466B
:100470000399D8400914731819055118039A384381
:10048000D2075140AC4009D00122944006D300224B
:10049000401C5141002C01D1400840001E4A9342AB
:1004A00012D3012203989206904207DB05204007F1
:1004B00009181A480143C012414004E003204007D4
:1004C0000818C10FC907002009B0F0BD0020F107CE
:1004D000FAE705180C464C4111486D42A04115D36E
:1004E00094181A465A410E48644290410ED3012096
:1004F0004A004005824209D35A00824206D359403D
:10050000C90F084AC90700201143DDE7002006494A
:10051000DAE700000000FF07FE070000FFFFFF7F93
:100520000000E0FF0000F07F0000F87F0121C90516
:100530000123411842001B06D3185B0E0AD0C110DC
:100540000722D206891840075242D14201D55200F3
:1005500089187047090208D50146002A03D0C10F47
:10056000C9070020704710467047420202D00020A1
:1005700002497047072109050143F4E70000F87FAD
:10058000F0B5FF252D04C609C209FF2704462E40F9
:100590000137CB093E4348402A402B400746002AFA
:1005A0006BD0002B69D0AA4267D0AB4265D000283F
:1005B00000DA32460125ED0529432C4309022002C9
:1005C000090AD21A4B0C7F24E31A434C000A7C44DC
:1005D000E35C7D242404121914145B00A2188842E1
:1005E00001D3521C00E0400049420C465C432411F8
:1005F0005C43DB016415E318040A5C43C502200D6B
:100600000C4644436419250A5D432303EC0C0D4654
:10061000654300030019EB184C42A34201D35B1859
:10062000401CD4052018002B07D05B00C91804D348
:10063000401C002901D1400840003F2189048A4222
:1006400009D3002A08DC1106090F04D00321490749
:100650004018C00FC007F0BD0122410012068918E2
:100660007F2252069142F6D205214907C84201D5A0
:100670009010F0BDFF20C005F0BD002F00DA32461B
:100680001648AA4207D2AB4205D21902090E17D06A
:10069000F80FC007F0BDFF2563002D06AB42F9D867
:1006A0004900A942F6D8AB4201D1A942F2D0A942F1
:1006B00001D1002101E061004908D0050843F0BDE7
:1006C0001102090EFBD0FF200243D005F0BD0A46FF
:1006D0000146104654E70000724300000000C07F4E
:1006E0000102C21504D00123DB071943002A0ADBEB
:1006F0009E239A1A02D40846D0407047FF22410038
:100700001206914201D900207047C017C0437047BC
:100710001F22030C02D10F2200041CD0030E01D1B2
:100720000002083A030F01D10001121F830F01D10B
:100730008000921E002801DB4000521ED205511895
:10074000021251181922904004D3491C002801D1EB
:100750004908490008467047C10FC90700D0404208
:10076000012292071143D3E701218907D0E7000056
:10077000F8B5264C4E00069DA6420AD8A64201D1E5
:10078000002806D15E00A64203D8A6420AD1002A5C
:1007900008D00D242404254233D02946002000F03F
:1007A00090F8F8BD0C461C4311D4994207D0C81AE2
:1007B00002D3EFF30080F8BDEFF30080F8BD801A9C
:1007C00002D3EFF30080F8BDEFF30080F8BD0924F9
:1007D0002407E5008B4207D0581A02D3EFF30080BC
:1007E00006E0EFF3008007E0101A03D3EFF3008078
:1007F000A04303E0EFF30080A043284380F3008888
:10080000F8BD009500F074F8F8BD00000000E0FFAE
:1008100010B5FF231B0644009C421DD84C009C428F
:100820001AD80346124A0B4307D4401A02D3EFF3F7
:10083000008010BDEFF3008010BD081A03D3EFF362
:100840000080904305E0EFF3008001219043C90749
:10085000084380F3008810BD0D231B041A4204D006
:100860001146002000F02DF810BD00F04BF810BD2F
:1008700000000090754600F04DF8AE460500694650
:100880005346C008C000854618B020B5FFF796FC57
:1008900060BCB64600260027C0C5C0C5C0C5C0C5DF
:1008A000C0C5C0C5C0C5C0C5403D490849008D464A
:1008B000704710B50446C046C0462046FFF751FCBD
:1008C00010BDC80212D54803400F002804D0C80349
:1008D000C043012188407047EFF300800001000908
:1008E00003210907084380F3008870470020704700
:1008F00010B500200249029A00F010F810BD000067
:100900000000F87F10B5024800F008F810BD0000A4
:100910000000C07F004870479800002010B50C46CA
:100920001107090F092904D00A290AD008290CD176
:1009300004E011460820FFF7C4FF06E0510606D583
:1009400001E0510601D50120C007214610BDD106A6
:1009500007D501010909CC084907000E0006044328
:1009600009E0410F20024907000A0143200E00065A
:100970001D22D14101430846E7E700000149182044
:10098000ABBEFEE726000200704770B514460D4668
:100990000646200407D0B0B200F006F82870641EA6
:1009A0006D1C761CF5E770BD70B5044600F0D8F8F4
:1009B000A020214DA847214EB047200AA847B047A4
:1009C000E0B2A847B04700F0CBF8A120A847B04755
:1009D000002000F037F9044600F0E2F8204670BD30
:1009E00070B514460D460646200407D02978B0B2EB
:1009F00000F006F8641E6D1C761CF5E770BD000063
:100A0000F8B50C46054600F0ABF8A0200A4EB047FA
:100A10000A4FB847280AB047B847E8B2B047B847C6
:100A20002046B047B84700F0BBF80A20F8BC02BC2B
:100A30008E4600F083B8C046A90C00080D0D0008D2
:100A400080B500F013F800F0B9FF01F0CBF801F029
:100A500021F801F091F800F05FFF00F0EDFF00F0E9
:100A600015FF80BC01BC864601F04AB8F8B50020ED
:100A7000022101F05BFB0A2000F060F8664D287946
:100A8000411973268C5D00F0B1F8844208D17420BE
:100A9000285C00022946743149784018286301E037
:100AA0000120687101240221204601F03FFB0A2049
:100AB00000F044F8287941198F5D00F097F88742DB
:100AC00008D17420285C0002294674314978401806
:100AD000686300E06C711320022101F027FB0A20FB
:100AE00000F02CF8287941198E5D00F07FF88642DD
:100AF00008D17420285C00022946743149784018D6
:100B0000A863F8BD6C71F8BD80B5C54841F200011D
:100B100002F065F8411E884180BDC04674223E48FF
:100B200000217E2A02D08154521CFAE78170018094
:100B30007047C0462C4800214170704781B000903A
:100B400003480099016001680029FCD101B0704799
:100B50003C0C002081B00090009801B0704700006C
:100B6000F8B501F0CFF8E44C01262046314602F0FA
:100B700032F802252046294602F02DF8042738468F
:100B8000FFF7E8FF2046314602F023F83846FFF72A
:100B9000E1FF20462946F8BC04BC964602F019B88D
:100BA000F8B501F0AFF8D44C02252046294602F0F2
:100BB00010F801262046314602F00BF8042738468B
:100BC000FFF7C8FF2046294602F005F820463146C7
:100BD00002F001F83846F8BC02BC8E46FFF7BABFF7
:100BE000014840787047C046F8000020B0B5401E6C
:100BF0000021094B74240A46CDB2A84204DD5D19D8
:100C00002D5D5219491CF7E70C4801788918407886
:100C10000918FF208843B0BD2401002010B5401EF4
:100C20000021064B0A46CCB2A04203DD1C5D12191E
:100C3000491CF8E7FF20904310BDC046400C00203F
:100C4000FEE70000FEB5009001F056F800210226F4
:100C5000012001900C46019D07291CD8A64F38465B
:100C60000291314601F0B5FF3046FFF773FF384679
:100C7000314601F0B0FF3846294601F0B0FF274663
:100C800004462846FFF766FF0299601E84417800FB
:100C90000419491CE0E7009810B100F0EFFF01E0F3
:100CA00001F00CF8E0B2FEBDFEB5044601F02AF8F2
:100CB00091480226314601F08CFF00270120019067
:100CC000072F1FD860B2002802948B4D284603D40A
:100CD000019901F07EFF02E0019901F07CFF3046AE
:100CE000094CA0472846314601F075FF3046A04721
:100CF0002846314601F06DFF3046A0477F1C029C1C
:100D00006400DDE7FEBDC046550B000870B500F07D
:100D1000F3FF794C0221204601F05DFF01252846B2
:100D2000FFF718FF00262046294601F058FF30B192
:100D3000701CFA2E0646F6D3FFF732FF04E00221BC
:100D4000204601F046FF0025284670BD00F06AB835
:100D5000FEB5A94802F0E6FE0920C6060121019170
:100D60000025202730462A463B46A44CA0470322B4
:100D70000292A34C304629463B46A04730463946AE
:100D8000A04A90471027304601992A463B469B4C83
:100D9000A04730462946029A3B46994CA047304628
:100DA0003946984A90474027304601992A463B46A3
:100DB000924CA04730462946029A3B46904CA047A9
:100DC000304639468F4A90478027304601992A4657
:100DD0003B468A4CA04730462946029A3B46884CFF
:100DE000A04730463946874A90478348401C02F066
:100DF00099FE854E3046019C21462A4623467F4F68
:100E0000B84730462946029A23467D4DA8473046CA
:100E100021467C4A03B0F0BC08BC9E461047C04641
:100E200000040048F8B51C4802F07CFE1B4F012569
:100E30000024724E38462946224642F20003B0474B
:100E40006F4E38462146224642F20003B0473846EC
:100E500042F2000101F0BDFE0F48C01C02F062FE2C
:100E6000254E3046294622462B46644FB847304629
:100E7000214622462B46624FB84702273046294674
:100E800022463B465D4DA8473046214622463B461A
:100E90005B4CA047F8BDC0461305000000080048A1
:100EA000F8B5E14CA34D2046A847601CA847601D3B
:100EB000A847114E002401258023504F304621467B
:100EC0002A46B8474023304621462A46B8470920DB
:100ED000C606304621462A4641F20003B84730464E
:100EE00021462A4640F20013B847F24821462A46D6
:100EF00048F20003B847F8BD00140048B0B50D48EB
:100F000002F010FEEB4C0121002520462A4640F657
:100F1000000301F069FE03222046294640F6000343
:100F200001F081FE204640F60001B0BC04BC9646AC
:100F300001F04FBE1205000070470000F0B585B00B
:100F4000D94C204602F0EEFD601C02F0EBFD0920BA
:100F5000C40601260227D64D204631463A4648F2BD
:100F60000003A8470021039103220492244D204648
:100F700048F20003A847204648F20001214A904762
:100F8000CC4808250296314601973A462B46C84C74
:100F9000A047C8480399049A2B46194CA047C54C52
:100FA00020462946174A90471025204631463A46A2
:100FB0002B46BF4EB04720462746039E3146049A33
:100FC0002B460F4CA047384629460E4A904720250D
:100FD00038460299019A2B46B54CA047384631460F
:100FE000049A2B46064CA04738462946054A05B0C8
:100FF000F0BC08BC9E46104711050000E92B000814
:10100000272C0008D32B0008000400480C48006877
:1010100040F2E831B0FBF1F0401E010E00D0FEE7D7
:101020000849094A5060094803680B4003218907B1
:101030005918016000209060072010607047C0467A
:1010400010000020FFFFFF0010E000E020ED00E0B6
:10105000F0B587B03648002141600E4601919349B2
:1010600040F210608847344D34492846884703AC25
:101070003349204688474720029020803148059018
:101080000496314A28462146904701272F4A284690
:10109000394600979047142002212D4A90472D4948
:1010A0002846884740F21060401C804988472A4EF5
:1010B00030462249884703AD28462149884702988F
:1010C000288020480590019C0494304629461E4AF9
:1010D0009047304639461D4A90471520032529463A
:1010E0001B4A904730461B49884740F21060801CDD
:1010F0006E498847194E30461049884703AF384635
:101100000F498847164838801648059004943046A1
:1011100039460D4A9047304600990C4A90471620B0
:1011200029460B4A904730460A49884707B0F0BD28
:10113000F8000020253B000800400140C13C0008A9
:101140000D3E0008E7030000353D0008E93D0008BA
:10115000293900082B3D00080044014000480140A7
:101160001F1C00000F270000FEB502901C20022566
:10117000294602F0D9FB4C4802F0D4FC0920C706EE
:1011800001240426019638462146324601F0F6FC39
:10119000384629462246334601F026FD00210091BB
:1011A00038462246334601F03EFD082638462146A1
:1011B000324601F0E3FC384629462246334601F028
:1011C00013FD3846009F39462246334601F02BFD79
:1011D000164802F0A7FC164D284602F06DFE284680
:1011E000029902F037FE2846394602F0DFFE284613
:1011F00041F2000102F0EFFE284640F2004102F009
:10120000C0FE2846019902F0C9FE2846314602F088
:10121000DAFE284602F06AFE0521284603B0F0BC3B
:1012200004BC964602F080BE1105000011070000C4
:1012300000440040F8B51C4C1C4D2046A847641CD7
:101240002046A8472046A8470920C5060126184C75
:101250002846314632463346A04700240327284615
:1012600021463A46334601F0DEFCA04802253146CD
:101270002A4644F200030E4EB0479C4E30462146AB
:101280003A4644F2000301F0CEFC304621462A469D
:1012900041F20003064CA047304644F20001F8BC7E
:1012A00004BC964601F097BC11050000253B0008E0
:1012B000E92B000800040048F8B500F01FFF0A24DD
:1012C0000F4E2046B04700F0E7FE2046B047002012
:1012D00002250C4A0C4F2946B8472046B04701204A
:1012E00029460246B8471320084A2946B8472046EF
:1012F000B04700F0E9FEF8BC01BC864600F008B833
:101300003D0B0008040A000051210008650400009C
:10131000FEB57020022100F009FF3220FFF70EFC1D
:101320006D4E3079811973240D5DFFF75FFC8542A6
:1013300007D17420305C000231467431497840187E
:10134000B0607120022100F0F1FE3220FFF7F6FBC1
:10135000307981190D5DFFF749FC854207D1742072
:10136000305C00023146743149784018F0607220D8
:10137000022100F0DBFE3220FFF7E0FB307981191B
:101380000D5DFFF733FC854207D17420305C00020D
:10139000314674314978401830610221204600F00E
:1013A000C5FE3220FFF7CAFB307981190D5DFFF7CA
:1013B0001DFC854207D17420305C00023146743137
:1013C00049784018706174250221284600F0AEFE6D
:1013D0003220FFF7B3FB307981190F5DFFF706FC70
:1013E000874206D1705D0002314674314978401859
:1013F000B0617520022100F099FE3220FFF79EFBBC
:10140000307981190F5DFFF7F1FB874206D1705DDE
:1014100000023146743149784018F061762002218B
:1014200000F084FE3220FFF789FB307981190F5DCF
:10143000FFF7DCFB874206D1705D00023146743154
:101440004978401830627720022100F06FFE322088
:10145000FFF774FB307981190F5DFFF7C7FB8742F7
:1014600006D1705D000231467431497840187062CF
:101470006F20022100F05AFE3220FFF75FFB307927
:1014800081190C5DFFF7B2FB844208D1705D000248
:1014900031467431497840180290B06201E0B06A78
:1014A0000290B068019037460C37BCCF306A00908C
:1014B000716A01988218D21812195219D21900981B
:1014C00010184018401E80B204494140F162029851
:1014D000091A48424841FEBD24010020FFFF0000D8
:1014E000E94840F6000101F078BBC046000400481E
:1014F000094A1018C9B24A07D20F02718A07D20FDF
:1015000042700A07D20FC271CA06D20F82728906D0
:10151000C90F41737047C0460000002070477047F4
:10152000F0B58BB00020B64C0490214640F29012EA
:10153000FFF72BFA0894207808B1042802D3B049A9
:1015400003200870AF49087040F2F810AE490858FF
:101550000A9040F2F4100858099040F2F0100A582E
:1015600040F2EC10085840F2E8140C590B25EE43F9
:10157000019608361827DEB1A1498D19697DB94059
:10158000234604460A9808180A9020461C46697C9F
:10159000B940099BCB180993697BB9408A18697ACD
:1015A000B94008186979B9400C19083F761CE2E780
:1015B00040F2F811944E0A9F775040F2F411099DC1
:1015C000755040F2F011725040F2EC11705040F240
:1015D000E813F4508D4E642C01D3B44201D98A49EA
:1015E000CE50642802D38949884204D940F2EC10D5
:1015F0006421854C21508648824204D940F2F01083
:101600008149834B0B508348854204D940F2F41042
:101610007D49804A0A508048874204D940F2F81038
:1016200079497D4A0A500498032872D004908000BA
:101630007549401840F2BC2142580A9240F28C246D
:101640000259099240F25C25435940F22C27C659B1
:1016500040F2FC128258411803910119029141197C
:101660000591C1190791114640F2FC1280180690AD
:10167000019F08371824E7B108460899CD19D921E8
:10168000695CA1400A9A8A180A92A921695CA14062
:10169000099A8A1809927921695CA140CB184921DD
:1016A000695CA1408E19697EA1400918083C7F1C25
:1016B000E1E7079806600698016005980360099FB6
:1016C000029D2F600A9A039C226064294F4801D32F
:1016D000814201D906990860642E01D3864202D95D
:1016E0006420079908604A48834202D9484805990E
:1016F000086048488742049801D94649296046490C
:101700008A4201D9444921600899091D0891401C69
:101710008AE740F205103A4D285C40F2F4213A4A3B
:10172000505040F2F8201018019FB91D40F20C12E1
:1017300021B16B189B5C08C0891CF9E740F21810B6
:10174000285C40F21C31304A505040F240301018B2
:1017500040F21E11691803238BB10C7804600A7BD8
:1017600002630CB1642C01D3012404600AB1642A21
:1017700001D301220263491C001D5B1EECE740F20D
:1017800027102A5C40F264311F4C625040F2331043
:10179000285C40F29433E0500AB1642A02D301225B
:1017A000194B5A5008B1642804D340F294300121F7
:1017B000154A115040F24315194E0021EFB1174858
:1017C000C21910693C460E4BDF1940F24013FB5C16
:1017D0001B06181840F24113FB5C1B04181840F25A
:1017E0004213FB5C1B0218187B5DC018B0420F4609
:1017F00000D807461761271DE0E70BB0F0BDC046D3
:10180000AC080020000000207C020020B01E040074
:101810008038010080B14F0100562183580200201A
:1018200000E1F50570B5154C8021154E2046B047F6
:10183000144D287040212046B04768700920C40626
:10184000204641F20001B047A870204640F2001146
:10185000B047E8700C4848F20001B0472978090108
:1018600001436878C0000843A97889000143E878FB
:1018700042000A431F20904370BDC0460014004838
:101880006F1C0008A20100200004004870B522204F
:10189000022100F04BFC0A20FFF750F9F04E30799E
:1018A000811973228C5CFFF7A1F984420AD174205C
:1018B000305A000400BAFEF757FFFEF737FE044621
:1018C0000D4603E00120707100242546F06E0D499D
:1018D00002F0A1FE08B90D4A00E00B4A08B90D4B11
:1018E00000E00B4B20462946FEF7FCFCFEF7BCFC53
:1018F0003067306D3F21090602F077FE08B90020FD
:10190000306770BD00005C42CFF753E34E62105861
:10191000A59BB43F39B4B83F70B52820032100F02F
:1019200005FC0A20FFF70AF9CD4D287941197324E7
:101930000E5DFFF75BF986420BD17420285C000432
:10194000294674314A781202101889784018A8651F
:1019500001E0012068710220014600F0E7FB0A2047
:10196000FFF7ECF8287941190C5DFFF73FF9844245
:1019700008D17420285C0002294674314978401847
:10198000E86501E001206871A86DFEF7EDFE0446F0
:10199000286AFEF7E9FE0146204602F013FF3121D6
:1019A000090602F00FFFB04C214602F00BFF214662
:1019B000FEF7E6FD2866686670BDC046B0B5242017
:1019C000032100F0B3FB0A20FFF7B8F8A44D2879F3
:1019D000411973228C5CFFF709F984420BD1742002
:1019E000285C0004294674314A781202101889785C
:1019F0004018E86302E001206871E86B010218D426
:101A0000FEF7B2FE0446A868FEF7AEFE0146204689
:101A100002F0D8FE0D21890602F0D4FE924C214638
:101A2000FEF7AEFD214602F0CDFE2146FEF7A8FDF1
:101A300000E000202864B0BDB0B52320022100F0F2
:101A400075FB0A20FFF77AF8854D28794119732232
:101A50008C5CFFF7CBF884420BD17420285A000429
:101A600000BAFEF781FE4121090602F0ABFE0146F5
:101A700002E00120687100210548FEF781FD04465F
:101A8000784902F0BDFD00B10024AC66B0BDC0468F
:101A9000647A5A4AB0B52C20042100F047FB0A2092
:101AA000FFF74CF86E4D2879411973228C5CFFF7D3
:101AB0009DF8844203D1686F00BAE86402E0012017
:101AC0006871E86C0121CA070021904200D9C9431E
:101AD0004840FEF749FE04466869FEF745FE214688
:101AE00002F070FE0321090702F06CFE5E4C2146F5
:101AF00002F068FE2146FEF743FD2865B0BDC046F2
:101B000070B52720032100F011FB0A20FFF716F81B
:101B1000534E3079811973228C5CFFF767F8844249
:101B20000AD17420305C0004314674314A781202C4
:101B300010188978441801E001207071306DFEF7AB
:101B4000F5FC0A4A0A4B02F045FD05460120C10595
:101B50008C4201D90006041B2046FEF705FE05490C
:101B6000FEF70EFD05B10020F06670BD3333333350
:101B70003333D33FFEFFFF4AB0B52E20042100F0DF
:101B8000D5FA0A20FEF7DAFF354D2879411973227C
:101B90008C5CFFF72BF8844203D1686F00BAE864CD
:101BA00002E001206871E86C0121CA07002190421F
:101BB00000D9C9434840FEF7D7FD04466869FEF7DF
:101BC000D3FD214602F0FEFD0321090702F0FAFDD4
:101BD000254C214602F0F6FD2146FEF7D1FC686552
:101BE000B0BDC046B0B52620032100F09FFA0A2000
:101BF000FEF7A4FF1A4D2879411973228C5CFEF779
:101C0000F5FF84420BD17420285C0004294674310E
:101C10004A781202101889784018686402E001209E
:101C20006871686C010218D4FEF79EFD04462869AD
:101C3000FEF79AFD0146204602F0C4FD6921C90560
:101C400002F0C0FD0749FEF79BFC074C214602F05D
:101C5000B9FD2146FEF794FC00E00020A864B0BD69
:101C6000240100200000C84200007A44704780B57B
:101C700000F0B5FF411E884180BD000070B52D4CBD
:101C800002250D4E20462946B04700F03BF80121C1
:101C90002046B0472846FEF75DFF2046294600F063
:101CA0009AFF2846FEF756FF20462946324670BC6A
:101CB00008BC9E461047C046D32B0008B0B51D4C4B
:101CC00002252046294600F084FF00F01BF8012180
:101CD000204600F080FF2846FEF73CFF20462946BC
:101CE00000F079FF2846FEF735FF20462946B0BCB4
:101CF00004BC964600F06DBF0E48002101230A4641
:101D000000F072BF70B50B4C00250126204631460D
:101D10002A46334600F068FF032220462946334610
:101D200000F081FF044848F2000170BC04BC9646F4
:101D300000F04FBF0014004800080048F8B5044602
:101D40000027CE4D084EA7420CD0EB48C15D284677
:101D500002F0ACF82846314602F0D5F80028F9D058
:101D60007F1CF0E7F8BDC046060700000348016885
:101D700011B10168491E01607047C0463C0C00204B
:101D800030B43348026801210A43026002689207B6
:101D9000FCD542682F4B1340436042682E4B1340E2
:101DA000436002682D4B13400360C26A0F239A43BD
:101DB000C262026B40F203139A4302630A04036B8C
:101DC00093430363CA07036B93430363426B8A43E2
:101DD00042630022826002680A430260204B0222B2
:101DE00004685D1E9D4202D214402B46F8D0036861
:101DF0009B0700D4FEE71B4B1C680725AC431C6007
:101E00001C6814431C604368436043684360436834
:101E100043604368144C1C4044604368134C1C43AB
:101E200044600B0604681C43046003689B01FCD5F6
:101E300043680324A34343604368134343604268F9
:101E40001207FCD5C806002130BC01F0A1BDC04678
:101E5000001002400C00FF08FFFFC277FFFFF2FEF8
:101E6000FF04000000200240FFFFC2F7000004084A
:101E700010B50A4C0121204601F0BEFF68B10121D6
:101E8000204601F0B5FF0021204601F017FF04486D
:101E9000006810BC02BC8E46004710BD0020004008
:101EA00014020020F8B51C4D01242846214601F0FB
:101EB000A3FF012803D10121284601F099FF3649EB
:101EC00020310022154B164D032A10D09E5C5EB1C6
:101ED0000E460C3E37680868874201D2781C02E043
:101EE000AC54002098543060091D521CECE70D4999
:101EF0000878294B58B19A68D868824202D2501C9F
:101F0000986004E0084804700020986008705968E0
:101F100009B1481E5860F8BD004001404102002050
:101F2000440200202F0200203002002010B5074C90
:101F30000121204601F060FF012806D10121204641
:101F400010BC04BC964601F053BF10BD00440140D4
:101F5000B0B5104D01242846214601F04DFF01285F
:101F600003D10121284601F043FF0B4801780229E3
:101F700001D8491C02E009490C7000210170016977
:101F8000782902D106490C7000214470491C016176
:101F9000B0BDC04600480140F800002028020020E3
:101FA00035020020B0B51D4C354D2046294601F0C4
:101FB000D9FF30B11A48006880472046294601F011
:101FC000BDFF184D2046294601F09DFF012806D18E
:101FD0002046294601F08FFF114800688047124DC6
:101FE0002046294601F0BEFF30B110480068804706
:101FF0002046294601F0A2FF0D4D2046294601F05A
:10200000B1FF48B109480068804720462946B0BC66
:1020100004BC964601F092BFB0BDC04600380140F6
:102020000C02002003070000070007071002002031
:1020300006000607B0B5114C114D2046294601F0A7
:1020400091FFD0B12046294601F078FF0D48007875
:102050000D4D297881420BD2204601F023FF2978CB
:102060000B4A50540B4801220270481C2870B0BD26
:1020700000202870054801210170B0BD00440040D7
:102080000500050728010020260100202501002069
:102090009801002024010020B0B5404800210171C2
:1020A0000424C4703C4D5A20A870EA206870A52012
:1020B00028702046FEF7B2FDE8702046B0BC02BC96
:1020C0008E46FFF73BBEC046B0B5344800210171D3
:1020D0000424C470304DDC20A870EA206870A5206C
:1020E00028702046FEF79AFDE8702046B0BC02BC7E
:1020F0008E46FFF723BEC046400C0020B0B52748EF
:10210000002101710424C470234DE520A870EA2049
:102110006870A52028702046FEF780FDE8702046F4
:10212000B0BC02BC8E46FFF709BEC04610B51A4AC5
:102130005070A5201070194C0220E070481C2071CE
:10214000FEF7ECFCE07810BC02BC8E46FFF7F6BD53
:10215000BCB5114BA5241C70802404435C70009214
:10216000981C6A46521E0C4624B1155D0570401C31
:10217000641EF9E7094800220271C91CC170CCB283
:10218000E018451E2046FEF749FD28702046BCBCDD
:1021900002BC8E46FFF7D2BD400C00202401002077
:1021A000B0B50020064CA047064D28600120A0478E
:1021B00068600220A047A8600320A047E860B0BD87
:1021C000FD390008A801002010B5144608463F4913
:1021D0000A220A700722214602F0A8F8012804D139
:1021E000044802F01DF9012801D0032010BD002091
:1021F00010BDC046204E0000F8B506460F4CA08822
:10220000000A16D1A0880527032810D30D46009296
:10221000A188264801F0E6FB48B9244908783070C7
:10222000481C2860A088801E009908800027384636
:10223000F8BD03A00C499C22FFF7C6FF1C0200203A
:102240007573526376427566666572506F73203C93
:10225000204D425F5345525F5044555F53495A45A4
:102260005F4D4158000000004D4C0008B0B5174DBF
:102270006B780BB1052516E00124EC804B1EAB609A
:102280001870E8888018E880E988184601F0AAFBF1
:10229000E9884A1CEA80054A5054AC70002528465B
:1022A000214601F0A5FE2846B0BDC0464A0C0020DC
:1022B00010B501200024214601F09AFE0348447025
:1022C000204610BC02BC8E4602F01EB81C02002044
:1022D00080B50020014601F08BFE80BC01BC864623
:1022E00001F0BABE10B5064C2078012805D105488A
:1022F000806880470020207010BD062010BDC046B9
:1023000014000020F4010020F8B50C4609880325CC
:1023100005292FD10279C17809028E18711E89B260
:10232000314B994226D8811C00918778417800254D
:1023300025800123037023885B1C23805307B2B2DE
:10234000D60803B1761C009B46702088401C208074
:102350000802C019401C81B218462B4600F0E8FA6A
:1023600020B1F8BC02BC8E4601F01CBBF0B2218843
:10237000081820802846F8BDF8B50C4609880325C2
:1023800005292ED10279C17809028E18711E89B2F1
:10239000154B994225D8811C0091877841780025FA
:1023A00025800223037023885B1C23805307B2B26D
:1023B000D60803B1761C009B46702088401C208004
:1023C0000802C019401C81B2184600F001FB20B180
:1023D000F8BC02BC8E4601F0E5BAF0B221880818BC
:1023E00020802846F8BDC046CE070000F8B50C4650
:1023F00009880325052923D10279511E7C291FD87C
:10240000831C81784778002525800326067026885E
:10241000761C2680560046702088401C208038029A
:102420004018401C81B218462B4600F0F7FA20B144
:10243000F8BC02BC8E4601F0B5BA20888019208015
:102440002846F8BDF8B50C4609880325052928D18A
:102450000179C278120251184A1E92B27B2A20D802
:10246000821C009287784378002525800422027020
:102470002288521C22808AB2560046702088401C56
:1024800020801802C019401C81B2009800F05CFB4B
:1024900020B1F8BC02BC8E4601F084BA20888019B5
:1024A00020802846F8BDF8B5054608880A2841D39B
:1024B0000C462879E97809020F18781E80B20326A5
:1024C0007C2838D8287AE97909020818411E89B28F
:1024D000782930D8697A82B2500081422BD1A8790C
:1024E000697909020818411CA87800906E7828467E
:1024F0000A3089B2012300F091FAB0B9BAB23002C1
:1025000000994018411CA81C0026268017232B7018
:1025100023885B1C238057006F7023885B1C2380FB
:1025200089B2334600F07AFA38B1F8BC02BC8E4664
:1025300001F038BA00263046F8BD2088C019208046
:10254000F9E70000B0B50C4605490D88401C891C10
:102550002A46FDF745FE681C20800020B0BDC0461D
:10256000C40100201CB50988032405291AD101796A
:10257000C1B982784378C178FF2900D091B9180297
:102580008018421C01A800244470FF394B424B4183
:10259000037091B20122134600F0CAF910B101F0A4
:1025A00001FA044620461CBD80B50988052910D1D2
:1025B0008178427812025118491C89B2C01C01224C
:1025C000134600F02BFA30B180BC02BC8E4601F0FD
:1025D000E9B9032080BD002080BD70B50C460A8893
:1025E0000321062A24D30679C27812029519AAB2C9
:1025F000D308760700D05B1C6D1EADB22D097A2D75
:1026000016D84579DBB29D4212D1817843781B02FE
:102610005918491C89B2801D012300F089F920B1A5
:1026200070BC02BC8E4601F0BDB90520208000219F
:10263000084670BDB0B50C460A880321062A20D38F
:102640000279437955062D0EAB421AD1C3781B028D
:102650009A18531E9BB2772B13D8817843781B02AC
:102660005918491C89B2801D92B2012300F0D6F995
:1026700020B1B0BC02BC8E4601F094B90520208088
:1026800000210846B0BD0000F8B50546022091B310
:10269000CC081E2C2FD8069C524E3170012D15D01F
:1026A0004DBB254D2548264FB760F0603561214868
:1026B00070611F48B0611D48F0611B4830620846D8
:1026C00011461A46234600F091F813E0134D1448C2
:1026D000144FB760F06035610F4870610D48B0610C
:1026E0000B48F06109483062084611461A462346F5
:1026F000FFF76AFD00B1F8BD01F000FE20B13848D7
:10270000012101700020F8BD0320F8BDC54100087B
:10271000FD410008B9400008F92100086D220008B9
:10272000D1220008B12200080945000855450008DB
:1027300079440008292800089D2800081D29000860
:10274000012900087CB52648007808B1062445E038
:1027500001A801F0C7FD002401283FD101A800789D
:10276000022812D0012839D11E4D6B69681C2946F8
:1027700024312A1D984788BB68782978884200D080
:1027800060BB022001F0C0FD28E0164D6A6A117896
:10279000A97000230120144C802B0AD0E65C46B1BE
:1027A0008E4201D00833F7E7E0184368291D104630
:1027B00098476978002489B158B10121A980A97886
:1027C00080220A43696A0A70A9884A1CAA806A6A38
:1027D0005054AA88696A28782B69984720467CBD9E
:1027E00014000020F40100201800002010B5144649
:1027F00008460822214601F099FD01280ED144F631
:102800000030844201D9232003E060000549B1FB78
:10281000F0F080B201F004FE012801D0032010BDC9
:10282000002010BDA07F1700F8B506460F4C608849
:10283000000A16D160880527042810D30D4600929F
:1028400061882E4801F0ECFA48B92C4908783070BC
:10285000481C28606088C01E009908800027384600
:10286000F8BD03A00C499C22FFF7AEFCE801002054
:102870007573526376427566666572506F73203C5D
:10288000204D425F5345525F5044555F53495A456E
:102890005F4D415800000000EF4B0008B0B51E4DE1
:1028A0002B78012B26D10124AC804B1EAB60187015
:1028B000A8888018A880A988184601F0B1FAA988CC
:1028C0004A1CAA800D4A5054A9884B1CAB80000AB0
:1028D0005054A868007801F099FDA888401EA8808F
:1028E000A868401CA8606C7000252846214601F0AD
:1028F0007FFB00E005252846B0BDC0464A0C0020FD
:1029000080B5054800210170012001F071FB80BCF9
:1029100001BC864601F0B8BBE801002080B500206C
:10292000014601F065FB80BC01BC864601F094BB0A
:10293000FEB514460246491E88B20019042824D860
:10294000601E0825019590FBF5F0451C0020F3B1B1
:10295000012B1BD100901D4B280435D06D1E029217
:1029600010782246019F541E12040BD03A0609D05B
:10297000012202408EB29A55491C7F1EC0B2400807
:102980002246F0E7029A521CE6E70120FEBD0090C5
:10299000082001900D4F280416D002926D1E0026CB
:1029A00022460198541E12040AD0020608D08AB2A8
:1029B000BA5CB2401343761C491C401E2246F1E724
:1029C000029A1370521CE6E70098FEBD4A0D0020E3
:1029D000F0B5491E8BB2DC0801217D2C1BD39B185E
:1029E00040F2EC34A34216D8511E082391FBF3F1B8
:1029F0004C1C002125040ED0641E16461D46721E76
:102A0000360404D06F1E2D0616463D46F7D100252C
:102A10000570401CEEE70846F0BD0000FEB5054617
:102A2000481E87B2012002904148874217D91446B8
:102A3000BE18404A964212D841F27072BE1A3E4AFF
:102A40005660012B0DD033BB401C87424AD1022C6B
:102A500048D170003B490968384A115252E0029847
:102A6000FEBD019654700520C04340F2D07343432D
:102A70003248C0187B00C3182746164638040CD0CD
:102A80002878000218806A78801832461880AD1CB9
:102A90009B1C7F1EF2E70020FEBD41F2EB70081A7E
:102AA00080B26B2802981CD801984000234909186D
:102AB0001078029047012248C5192846083022069E
:102AC000D20DFDF78DFB01201D49C85101986860AA
:102AD0000298411CCAB200200F2A024600D80A46BA
:102AE0003270FEBD41F2EB70081A793080B2E728EF
:102AF0000AD8700011490818B100124A5118620032
:102B0000FDF76EFB002000E001200521CA4340F2E2
:102B1000D0715143094A5218790051182204E0D06B
:102B20004A782A700A786A70AD1C891C641EF5E721
:102B30006F170000581B0000B80100204E0D002048
:102B40003C0A00207C02002010B50346481E81B2DA
:102B50000120084CA1420BD38918074CA14207D889
:102B60000020110404D0587018709B1C521EF8E706
:102B700010BDC046B80B0000BC0B0000FCB50191B5
:102B8000016A0090446A00252E46202D0CD017467D
:102B9000F740FF0705D0019FAF400F23AB4099439B
:102BA00039432D1D761CF0E708250026202E0CD079
:102BB0001346EB40DB0705D0019BB3400F27B7401E
:102BC000BC431C43361D6D1CF0E700980162446253
:102BD000FCBD8162704781617047C16270470069C6
:102BE0000840411E88417047FEB502930192026879
:102BF0000090C56800263746202E10D0029BFB406F
:102C0000DB0709D0019BB3400324B440A5431D4317
:102C10000B46B340A2431A43B61C7F1CECE7009856
:102C20000260C560FEBDF8B5012902D141681943B3
:102C300001E04168994341600090816800240320CD
:102C40002646202C0CD01F46F740FF0705D017461C
:102C5000A7400546A540A9433943A41C761CF0E7CC
:102C600000988160F8BD000000B59FB0E44A0027DD
:102C7000978257715770E3480321199101700B2017
:102C8000C0431A90093020B11118CF770F77401C3C
:102C9000F9E71772D771FFF773F8FFF781FAFEF7BC
:102CA0004BF9FEF7B3F9FEF729F9FEF7F9F8FEF74D
:102CB00045F9FEF7BFFAFEF7CBF9FEF747F8FEF746
:102CC0002FFC42F28050FEF74FFAFEF741F8092040
:102CD000C0060A9001244020049080201E902646C1
:102CE000C8480078844226D8032C09D0022C11D081
:102CF000012C1ED10A9D28460499FFF76CFF0EE0B7
:102D00000A9D28460499FFF766FF28461E99FFF79B
:102D100060FF08E00A9D28460499FFF75AFF2846FD
:102D20001E99FFF758FFB8483146FFF754FFFEF7EA
:102D3000C3FA641CD4E7FEF775FD01460097E12055
:102D4000430238463A46FFF79FFCFFF7CBFA40F2C2
:102D5000F4213846AD4F7B580499A94A5354AC49E5
:102D6000D18140F60001C91C396040F2B411795894
:102D7000403202925170D9B20546FEF7B9FB0121EB
:102D80000A980991FFF725FF2524282C19D0002047
:102D90009B4908554819791940F2F8268A59442365
:102DA000C25489198B6C46268355896F4723C154B9
:102DB000D1B220462438C0B2FEF79AFB2D1D641C08
:102DC000E3E740F21C3038582B2108918C4A5054CC
:102DD00007200D90C00340F2B411785000200590F8
:102DE000D07288481999017040F2943038581146D1
:102DF0002B31C87040F2643038588870108A508285
:102E0000099D28040C9068040B90824E824940F280
:102E100006100818039040F2B8103818079040F2D6
:102E2000341008180690FDF76FFE002800D02CE142
:102E30000898734E325C104628403073F17A88420D
:102E400003D10020B071317A28E050B90123B37268
:102E50000021717252B2002A16D433720022F2712C
:102E600010E0059BB3727572510604D435720022CE
:102E7000F27129460FE03372F5712D21725C40F238
:102E8000E8314A43194606E03172F3712E22B25CF2
:102E900040F2E8335A43F0726048026039B30024CC
:102EA0003472F471707A40B120215748FFF793FED5
:102EB00074720898315C01200AE0B07A60B1202178
:102EC0005148FFF786FEB4720898315C1A980A30B0
:102ED000084340F21C3178504B4C204644F200012C
:102EE000FFF779FE204644F20001FFF772FE002052
:102EF00016251D90192D00D1C3E0741933461E907C
:102F0000311844201C91095C012208461B92104094
:102F1000A074E27B824205D11E46585D90B300202A
:102F200070552FE01E46002240B962721B9B23732E
:102F300049B200291AD4E270A37122E022731B9FC8
:102F40006772490605D436491E9BCA50E270A771C4
:102F50000AE0E770A27146211C9A515C40F2E83207
:102F600051432F4A1E9BD150284F0AE0E370A271B3
:102F700047211C9A515C40F2E8325143284A1E9B7B
:102F8000D150E073A079002874D01C9E44360027ED
:102F9000A771E770607A58B17F201D990840022818
:102FA0001BD001281BD0F0B90A9848F2000118E0A4
:102FB000207B002851D01C9627737F201D99084044
:102FC000022816D001281B9E2CD0104C78BB0A98E2
:102FD00048F20001FFF7FDFD29E0102100E0082183
:102FE0000948FFF7F8FD677230781B990843074CD2
:102FF00020E010210448FFF7ECFD044C1B9E16E076
:103000002802002000000020000400487C0200206C
:10301000030800003C0A00201C07002004010020D7
:10302000180100200821F048FFF7D3FDEF4C1C9851
:103030000078B043294616391E9AA218C0B240F251
:10304000F823D050CAB2199BB2FBF3F25A43891A43
:103050003639CF220A4091006050E34C204644F2BA
:103060000001FFF7B8FD204644F20001FFF7B1FD73
:10307000DF4EDE4F6D1C1E98001D1D99491C1D91D1
:1030800038E700207080099DDA4EFFF75BFBFDF703
:10309000A7FD18B1FEF724FAFDF74CFDD449487B93
:1030A00000B3002048731A98A0B1D34909183A1800
:1030B000526B40F24313CA54130A40F242140B55A8
:1030C000130C40F241140B55120E40F24013CA5437
:1030D000001DE9E740F205102F300C220699FDF79C
:1030E0007FFCC3490878002800D139E200240C7025
:1030F000032C04D0E0B200F035FD641CF8E7BF4CAF
:10310000266A616AA06A1690206C1D90626CA06CA1
:103110001590256E606EA36E14937E601D9BBB6040
:103120001B95FD601391396112927A611190B8611B
:103130001698F86115983862AD4A343207CA1D46B0
:10314000A36B1B18A06D4118A06F8018149A7A62A7
:103150001093BB620F91F9620E903863AE4228461D
:1031600000D830461B9A904240F2B41300D8024671
:1031700001240021A24882421894204600D3084628
:10318000AE422A4600D332461B9C04B11B9A1C96C1
:103190009C4CA24200D81891189901401891FE1831
:1031A0009948407817900D25112D00D1C5E128468A
:1031B0000D38C0001E900D2D0FD1189808B39048FF
:1031C0001C99814203D2012040F2983178508C48FA
:1031D0001D9981421FD2012017E08B4840191A998E
:1031E000405CB0B31E980D3080B280003958B06C8E
:1031F000814237D930680121014302208143316087
:1032000040E0002040F29831785040F2A0317850F0
:1032100040F29C3178501798F8B140F2B41240F265
:10322000E8103858012100241C9B83420B4600D82B
:103230002346BA58199FBA43D3181D9A824200D820
:103240002146490059181B9A824215D9042001438E
:1032500014E03068012188430CE0F8580D99884348
:10326000F8500FE03068199A9043B26F914201D83C
:1032700002210843306005E0042081435B4F40F2A7
:10328000B413F950604840191A990C18E07890B1BD
:103290000D2D25D1384640F2EC117F58C0585B49BE
:1032A000303101401C9ABA423DD840F2E8308242A7
:1032B00036D9082036E00D2D1ED1FF58534807405F
:1032C00040F2E8301C99814202D848F200000743DE
:1032D00040F2E8301D99814213D80C98074312E060
:1032E0001E980D3080B2800039583068B26C91421F
:1032F00003D80221084302E030680221884330608D
:1033000033E04348074040F2E8301B99814202D93C
:103310004048074001E00B9807433448C75018E085
:1033200048F2000001433A48283008401D9ABA424A
:1033300007D840F2E8318A4201D9102100E00C9907
:1033400008433449183101401B9ABA4203D927482F
:10335000C150074609E040F2E830824201D92020FE
:1033600000E00B980143214FF950A07910B30D2DC7
:1033700028D13946FF58C020874340F2F010085842
:103380000123002213998142194600D81146890170
:103390007F181299814200D81346D9017918134A2F
:1033A00040F2B413D150119F874237D940F2001038
:1033B000014336E00D2D12D1F8581749263101404E
:1033C000F95030E0A82031581E980E3080B28000AD
:1033D0003A5830688A4203D90421084302E0306831
:1033E0000421884330601EE0000400487C02002075
:1033F000280200203C0A00201C0700207C06002038
:1034000030750000BFD4010000000020C77FFFFF1F
:10341000C7FFFEFFC7FFFDFF19FEFFFFEE48E630C6
:103420000140D150ED4F607A70B10D2D14D1F95893
:1034300040F20060814340F2F41038580024169A9C
:1034400082421BD823461AE00D2D12D1F85840F6BF
:1034500000618843F85029E0D82031581E980F3079
:1034600080B280003A5830688A4203D90821084364
:1034700002E0306808218843306017E001235A02D7
:103480008918159A824202D940F2E834183440F281
:10349000B4132143F950149A824203D940F6000034
:1034A000014302E040F600008143F950CC48405D02
:1034B00008B30D2D27D1FA5843F20000824340F2A1
:1034C000F410385801210023109C84420C4600D887
:1034D0001C46240312190F9C844200D81946490344
:1034E000511840F2B413F9500E9A82421ED944F298
:1034F000000001431DE00D2D13D1F85847F20001E3
:103500008843F85016E040F2081031581E981030E9
:1035100080B280003A5830688A4203D910210843AB
:1035200002E0306810218843306003E044F200007C
:103530008143F950361D6D1C36E6F448008A00219F
:10354000079A099DF54E032908D001238B4010CA24
:103550000CB1184300E09843491CF4E7EB4908829A
:10356000487941017258002A00D182E070184468FD
:103570007A2C77D321467A3904291CD88A0001A3F2
:103580009A18974600F008B800F02BB800F038B849
:1035900000F046B800F054B8806840F2E811785066
:1035A000DD4A1071010AD170010C9170000E50704B
:1035B000511C012053E08A2C03D9962C01D9A22C4E
:1035C00060D88068A1007850D24A8A18010ED24B88
:1035D00099549918C870030C4B70000A887090B207
:1035E0003DE0806840F2EC117850CB4A1072010A3D
:1035F000D171010C9171000E5071511D05202EE00A
:10360000806840F2F0117850C34A1073010AD172F9
:10361000010C9172000E50721146093109201EE012
:10362000806840F2F4117850BB4A1074010AD173DB
:10363000010C9173000E507311460D310D200EE0F8
:10364000806840F2F8117850B34A1075010AD174BD
:10365000010C9174000E5074114611311120042296
:10366000FDF7BEF9A94B58794101002272500121A2
:103670001971401CC1B20F2900D90020A34948711B
:10368000FFF7D1FBAE2C12D8A100A24A5218A24BD0
:10369000D31880683324185578503032010E9E4C70
:1036A000A154010C31241955000A322113E0BA2C1F
:1036B00015D8A100974A5218974BD31880686324F5
:1036C000185578506032010E934CA154010C6124BE
:1036D0001955000A622158548F4881187FE7BD2C84
:1036E00016D0BC2C2AD0BB2C52D10120874988701F
:1036F000894840F2061140184421502953D00278DD
:1037000041231343814A53540370091D801CF4E77D
:1037100080687E4C0499605440F205117E4A5054F2
:1037200040F2F4217850C1B240F20510FDF768F97B
:103730000498215C0020FDF7DBFE93E7012073492C
:10374000C8704420039950280BD00A787E23134078
:103750007F22D2439A186D4B1A540A70001D891C9F
:10376000F1E76D4C40F20610211840F20510401CA4
:103770000622FDF735F940F21812A05C7E210140C7
:103780007F20C04308180899604B5854A0541DE08E
:10379000C92C27D8017A2546BE3D092D69D1089844
:1037A0005A4A115473E05C4C40F20610211840F262
:1037B0000510401C0622FDF713F940F21812A05C18
:1037C000412101430898514B1954A154A11840F2CA
:1037D00005101330022243E719FEFFFF7C02002090
:1037E00000000020CF2C5FD88168CA3C1998604344
:1037F000421C9300029DE954871CBE00A955C01CC1
:103800001E9080001D9029544048001901238375A3
:10381000D0B2C9B2424A9047A95D404EF8B23C4F7F
:103820003F4A90471D98295C1E98C0B23C4A904779
:103830000620604340F200110C18A01D334949795D
:1038400049017118097A344A1154254608355155F1
:103850000A34115580B2334A90472F48415DA8B2CF
:10386000099D304A90472C48015DA0B22D4A9047EF
:10387000F8E6BD3CA000254A1018049A8154E0B235
:10388000FDF736FE21484079400130188168680014
:1038900040F200121018801D1F4A115480B2C9B2A4
:1038A000FDF7AEF8099DDDE6DB2C0FD882682046D7
:1038B0004E3019490A54D1B2A300F950D92C18D06E
:1038C000124C1B1940F2FA241B1B14E0E52C00D902
:1038D000C8E6806822464E320F498854C1B2A30020
:1038E000F950E52C0AD0094C1B1940F229341B1B56
:1038F00006E0064B2D331A7080B203E0034B2E33E3
:10390000187090B2FDF77CF8ACE6C04628020020A3
:103910007C02002019FEFFFF1C0700203C0A00204B
:10392000F1140008010A000870B540B2002817D44D
:10393000032302469A43144BD4588507ED0EFF2605
:10394000AE40B4438901C9B2A9402143D1501F21DF
:10395000014001228A40400980000C49425070BD5C
:103960008207D20EFF2494400F230340083B03201C
:10397000834304481D58A5438901C9B29140294396
:10398000195070BD1CED00E000E400E000E100E033
:10399000024A0A40024302480260704780FFFF1F4C
:1039A00008ED00E040B1072803D0012803D1022030
:1039B0007047062070470420704700000A2801D293
:1039C000302102E0102803D237210818C0B2704716
:1039D00002A0034940F2D012FEF7F6FB30000000CF
:1039E0004D4C000800220B0405D00378D218D2B247
:1039F000401C491EF7E75042C0B27047F8B5014677
:103A00003E4B18680C2202403D48082A044618D153
:103A10001A689202120F0F2A01D0941C00E01024A1
:103A20001D682D0101D5113214461A68D20301D444
:103A3000344A05E09A6A0F2515406A1CB0FBF2F281
:103A400054431D6818681A6805291FD800902D0670
:103A50002D0F2DA77F5D2546FD409204520F2E4F5E
:103A6000BE5C2A46F2408E0001A080198746C046FF
:103A700000F00AB800F011B800F00AB800F00EB873
:103A800000F00EB800F014B8224607E0002205E06E
:103A900000984005400F385CC5402A461046F8BDE6
:103AA000D86AC0051AD4D86AC00320D51C48F8BD0E
:103AB000D86A8007F2D0D86A03210840012822463C
:103AC000ECD0D86A084048F200020228E6D0D86A52
:103AD000084003280A4800D00020F8BD18680004F8
:103AE000800FD96A002904D4B2FBF0F2D6E70B4864
:103AF000F8BD401CB5FBF0F2D0E7C0460410024010
:103B000000127A0000093D000000000000000000E3
:103B10000102030406070809844B0008809FD500B2
:103B2000003FAB011F21014001228A4080090C495E
:103B300043581343435070471F21014001228A40DC
:103B40008009074943589343435070471F21014060
:103B500001228A4080090249435813434350704769
:103B600000100240FEB50446401C4F4FB871022CB5
:103B70000CD0012C16D0002C00D094E0029009202B
:103B8000C50640212846FFF726F812E002900920DA
:103B9000C50640212846FFF71EF880212846FFF77A
:103BA00018F80AE002900920C50640212846FFF7D0
:103BB00010F880212846FFF70EF83C480121FFF756
:103BC0000AF8FCF73DFFB86C394D294600F0FAFDC4
:103BD000FCF786FD1F2800D20020B9794901354A3B
:103BE00050505618386C294600F0ECFDFCF778FD73
:103BF00070601E2804D8301D0025056028460CE0A2
:103C0000386D2B4900F0DEFDFCF76AFD0546786D46
:103C1000274900F0D7FDFCF763FDE1000191306119
:103C2000B5606DB1386DFC6E2146FCF7A9FC796D6D
:103C300000F020FE1E4900F0C5FDFCF751FD01E03B
:103C4000FC6E0020F060B86E194D294600F0BAFDF8
:103C5000FCF746FD7061386E294600F0B3FDFCF7B5
:103C60003FFDB0612046294600F0ACFDFCF738FD71
:103C7000F061029840010F490A580292019AD2B2AB
:103C800092000D4BD2180818071DF8CF8169C06942
:103C90000190029850639363D463156456649764EB
:103CA000D16401981065FEBD240100200004004885
:103CB00000007A447C0600207C02002041627047AC
:103CC00010B5154C4449884213D01449884212D08B
:103CD000EC49884211D03D49884213D03D49884281
:103CE0000DD03E4988420CD03949884213D1F63470
:103CF00008E0E41D06E0F93404E0FD3402E0641D50
:103D000000E0A41D2046FFF721FF204610BC02BCA6
:103D10008E46FFF711BF10BD0B03000000100040DE
:103D200001680122914301607047016801220A4342
:103D30000260704710B50A888262244A904202D01D
:103D4000234B98420BD103687024A34303604B8834
:103D500004681C4304608B8804681C4304608B68FF
:103D6000C36290420FD1136840F20034A343136042
:103D7000CB8814681C431460097B016341690122EC
:103D80000A43426110BD124A90420BD0C94A904288
:103D900008D0104A904205D00F4A904202D00F4AF4
:103DA0009042EBD1026840F200339A430260CA8825
:103DB000036813430360074A9042DDD0074A9042EC
:103DC000DAD0054A9042D7D0D8E7C046002C01404F
:103DD0000004004000400140004801400044014010
:103DE000C2688A43C2607047C2680A43C2607047B3
:103DF00002698A4302617047C2680A40531E9A41B1
:103E000000690840411E8841104070470349002264
:103E100002730260426081607047C046FFFF00008D
:103E2000F0B5FF24094A0A4B25460E0409D006784E
:103E30007540565D5F5D25467D40401C491E3446F9
:103E4000F3E72002284380B2F0BDC046844A000850
:103E500084490008B0B50D4604467E48844204D02B
:103E60002048844205D1022000E00520FFF7C6FD6E
:103E700000E000202168090405D469084018B0FB5F
:103E8000F5F080B209E0690840004018B0FBF5F099
:103E9000034901400007400F4018E060B0BDC04634
:103EA000F0FF0000416A034808407047014A0A4099
:103EB00082627047FF01000010B56649884204D055
:103EC000084988420BD1084C00E0054C2046FFF71A
:103ED0003DFE204610BC02BC8E46FFF72DBE10BD35
:103EE0000E0300000044004011040000016801229C
:103EF0000A43026070471F220A4001219140026A72
:103F00000A43026270471F220A4089090958D140BA
:103F10000120084070471F220A400123934089096D
:103F20000A589A430A5070471F220A4001239340BF
:103F300089090A581A430A5070470000084A9142FA
:103F400006D1D021425848F200039A4342507047AC
:103F5000C902C90E01228A40016A114301627047F9
:103F600009340F341F220A400B049B0D1B58D34009
:103F70008A0D1258C802C00EC2401A4001201040DB
:103F80007047026801239A430260026840F20063AE
:103F90009A43026002680A43026070470268042381
:103FA0009A43026002680A43026070470268012374
:103FB0009A430260426843F200039A4342604268B7
:103FC0000A4342607047026808239A43026002680D
:103FD0000A4302607047026801239A430260026844
:103FE00041F200039A43026002680A43026070478C
:103FF00070B50E460921CC06CB4D0521012808D10C
:104000002846FFF791FF204640F60001FEF7E1FD4C
:1040100007E02846FFF77FFF204640F60001FEF745
:10402000DAFD06212846012E09D1FFF77DFF204643
:1040300040F6000170BC04BC9646FEF7CCBDFFF70D
:104040006AFF204640F6000170BC04BC9646FEF7AD
:10405000C0BDC04600380140B0B5164C0021204616
:10406000FFF72CFE012520462946FFF7C1FE20461A
:104070002946FFF7B5FE2046B0BC02BC8E46FFF7CE
:104080004FBEC04600200040B0B50A4C002120467B
:10409000FFF714FE012520462946FFF7A9FE20461A
:1040A0002946FFF7A1FE2046B0BC02BC8E46FFF7B2
:1040B0003CBEC04600200040BCB53A4DA878002860
:1040C0006AD101A800F028F96878002478B10228A4
:1040D00018D001285ED1FFF7D7FF01A800780D287E
:1040E00028D000243A2828D1EC70AC8052E001A8F6
:1040F00000783A284ED1FFF7C7FF0024AC80EC705F
:10410000012018E001A800782978884208D1FFF73B
:10411000A3FF00206870012000F0F6F8044639E0A3
:1041200000243A2810D1EC70AC8001206870FFF7B1
:10413000ABFF2FE0022068702CE001464139C9B284
:10414000062903D3E14303E06C7023E001463739CD
:104150003038C2B20A2A00D30846E97801290AD0C9
:10416000C1B9A988FF2911D8A9880001E54A50548E
:104170000120E8700EE0A988E24A535C03435354DF
:10418000A888401CA8800024EC7003E000246C7018
:10419000FFF762FF2046BCBD03A05149E322FEF7B2
:1041A00013F8C0461C02002065536E64537461749A
:1041B00065203D3D2053544154455F54585F494468
:1041C0004C45000080B53E484178491E012902D87F
:1041D0000021417005E04178012902D04078022891
:1041E00003D1FFF739FF002080BD03483C4940F26E
:1041F000A712FDF7E9FFC046094C000870B5304E24
:104200007078002856D1B078042840D8810001A2E7
:1042100051188F4600F008B800F027B800F009B830
:1042200000F02BB800F014B801200021FFF7E0FEE9
:104230002DE0F08830B3F07801282AD038BBB06880
:1042400000780009FFF7BAFB00F0E0F8012012E067
:104250000024B470032000F057F8054601202146E1
:10426000FFF7C6FEB470284670BD3A2000F0CEF8C5
:104270000220B0700020F07009E0307800F0C6F83D
:10428000042003E00D2000F0C1F80320B0700020EE
:1042900070BDB06801780F200840FFF78FFB00F079
:1042A000B5F80020F070B068401CB060F088401E87
:1042B000F080ECE703A00A4940F24F12FDF784FFBB
:1042C0001C020020655263765374617465203D3D85
:1042D0002053544154455F52585F49444C450000B7
:1042E0004D4C00080B490A78012A05D14A78027022
:1042F0000020087001207047002070470548002109
:10430000017001207047C0460249487001200870C2
:104310007047C046C001002010B504463F48FFF773
:10432000C1FD2070012010BD00380140FEB5029192
:104330001B2000252946FFF7F7FA3148FFF7F2FB6B
:104340000920C60601243046214640F20022FEF72D
:1043500015FC022101913046224640F20023294FEC
:10436000B847294F30462946224640F20023B84735
:104370003046214640F20042FEF700FC30460199EB
:10438000224640F200431F4FB84730462946224696
:1043900040F200431C4FB847304621462A4640F6BB
:1043A0000003184FB84703223046294640F6000361
:1043B000154EB0471248FD30FFF7B4FB174E30469C
:1043C000FFF77AFD30460299FFF744FD3046294653
:1043D000FFF7ECFD30462946FFF7FDFD3046294644
:1043E000FFF7CFFD04213046FFF7D8FD0821304606
:1043F000FFF7E9FD3046FFF779FD2046FEBDC046D8
:1044000011050000E92B0008272C000880B50146A3
:104410000248FFF74BFD012080BDC0460038014037
:104420007FB5054640F20870FFF77CFB104C204634
:10443000FFF746FC6E463046FFF7E8FC0D4830803B
:10444000681E02900020019020463146FFF772FC62
:10445000012520462946FFF7C7FC13202946FFF710
:1044600063FA2046FFF761FC284604B070BDC046E1
:10447000002000400F0E00001CB51A4C607858BB9D
:1044800001A8FFF749FF2078032823D8810001A263
:1044900051188F4600F01CB800F004B800F00CB8BA
:1044A00000F016B8002060806088411C61801549CA
:1044B000019A0A5402200AE06088FF2806D8608822
:1044C000411C61800F49019A0A5401E003202070C9
:1044D000FFF7DAFD00201CBD03A03D49F022FDF7E7
:1044E00073FEC046E801002065536E645374617426
:1044F00065203D3D2053544154455F54585F494425
:104500004C4500004A0C0020B0B5294D2878002405
:10451000032808D0022802D058B9002000E001206A
:10452000FFF7F2FE0446FFF797FD012028702046B2
:10453000B0BD28780028F6D028780228F3D0287853
:104540000328F0D00248224940F26512FDF73CFEF4
:104550008C4B000870B5164E3078012822D1707847
:10456000012805D080B901200021FFF741FD0BE0B3
:10457000B08858B1B0680078FFF748FFB068401CB9
:10458000B060B088401EB080002070BD0320FFF7EF
:10459000BBFE0446012000252946FFF729FD757062
:1045A000204670BD03A00A4940F22B12FDF70CFE15
:1045B000E8010020655263765374617465203D3DC7
:1045C0002053544154455F52585F49444C450000C4
:1045D000EF4B000810B500F029F8EFF300808000E1
:1045E00001D4012010BD002010BD10B500F096F8D8
:1045F000EFF30080800001D5012010BD002010BD28
:1046000010B500F08BF8EFF300804000800F012818
:1046100000D0002010BD10B500F0AAF8EFF3008024
:10462000800001D4012010BD002010BD70B501250F
:104630002D050C001C4310D4EC4206D4AC420AD425
:10464000994200D070BD904270BDE94217D4EB4250
:1046500015D4994270BD894270BDEC4206D5AC427A
:10466000F9D58B4200D070BD824270BD6D004C0008
:10467000EC4204D25C00EC4201D28B4270BD034C90
:1046800030B4FCF775F830BC70BD00BF19001604DB
:1046900070B50125ED0704004C4020D4441A01D226
:1046A000001B0919C60D4B00F2B2FF2A29D01B0EC0
:1046B0002CD000020C0228432C43D31ADC400519ED
:1046C00010D2280A02D3401C6D0611D0761EF605C2
:1046D0008019FF2A00DA70BDC00DC00570BD6940A9
:1046E00000F0CEF801200543C541521C761CE8E7D6
:1046F00064089C40C90161408900E7D10124A043BE
:10470000E4E71B0E440200D0034870BD002AFCD130
:10471000C00FC00770BD00BF0000C07F0123DB05D4
:1047200002000A430DD4DA4203D49A4207D48842E5
:104730007047D84214D4D94212D48842704780427C
:104740007047DA4203D59A42F9D5814270475B003F
:104750004200DA4204D24A00DA4201D28142704772
:1047600010B5024AFCF754F810BD00BF090013044D
:104770000123DB0502000A430DD4DA4203D49A4236
:1047800007D488427047D84214D4D94212D4884200
:10479000704780427047DA4203D59A42F9D5814288
:1047A00070475B004200DA4204D24A00DA4201D28A
:1047B0008142704710B5024AFCF72AF810BD00BFCD
:1047C0000900160470B5420064414B005C41120EB2
:1047D00039D01B0E38D0FF2A3CD0FF2B3AD0D2184C
:1047E0007F3A40024902400A490A4518ED01060095
:1047F0004E43000A090A48430104731A4019190C70
:104800004318990F04D05B08012149075B1A521C19
:10481000D80904D3401CF50301D19D0607D0FF2A17
:1048200008D2D50506D0E4072043401970BD012504
:10483000A843F4E7002A01DCE00770BD2402FF2052
:104840002043C00570BD1B0EFF2A03D0FF2B01D0F3
:10485000E00770BDFF2636064500B54206D84D007C
:10486000B54203D8D218FF2A00D0E7E7004870BD50
:104870000000C07F70B50125ED0704004C4022D434
:10488000441A02D26C40001B0919C60D4B00F2B24B
:10489000FF2A4BD01B0E50D000020C02A8432C4321
:1048A000D31ADC40051B05D5AD0019D36D08761E63
:1048B000521E37D0F605280A01D2801970BD70410A
:1048C0006D0603D070BD6940FFF7E8FE9C40090209
:1048D0006140490001D0401E70BD0124A04370BD5D
:1048E0006D081DD001202B0C01D12D0410302B0E92
:1048F00001D12D0208302B0F01D12D01001DAB0F6E
:1049000001D1AD00801CEB0F01D16D00401C361AA7
:10491000121A6D00680AF5054019012A02DB70BD04
:10492000002070BDC036300AC00770BD1B0E4402A7
:1049300001D1FF2B00D1024870BD002AF0D070BD1C
:104940000000C07F8182838485868788898B8C8DD7
:104950008E8F919293959697999A9C9D9FA0A2A3D2
:10496000A5A7A8AAACAEB0B2B3B5B7B9BCBEC0C219
:10497000C5C7C9CCCED1D4D7D9DCDFE2E6E9ECF0AB
:10498000F3F7FAFE00C1814001C0804101C08041BF
:1049900000C1814001C0804100C1814000C181400F
:1049A00001C0804101C0804100C1814000C18140FF
:1049B00001C0804100C1814001C0804101C08041EF
:1049C00000C1814001C0804100C1814000C18140DF
:1049D00001C0804100C1814001C0804101C08041CF
:1049E00000C1814000C1814001C0804101C08041BF
:1049F00000C1814001C0804100C1814000C18140AF
:104A000001C0804101C0804100C1814000C181409E
:104A100001C0804100C1814001C0804101C080418E
:104A200000C1814000C1814001C0804101C080417E
:104A300000C1814001C0804100C1814000C181406E
:104A400001C0804100C1814001C0804101C080415E
:104A500000C1814001C0804100C1814000C181404E
:104A600001C0804101C0804100C1814000C181403E
:104A700001C0804100C1814001C0804101C080412E
:104A800000C1814000C0C101C30302C2C60607C7FE
:104A900005C5C404CC0C0DCD0FCFCE0E0ACACB0B6E
:104AA000C90908C8D81819D91BDBDA1A1EDEDF1F9E
:104AB000DD1D1CDC14D4D515D71716D6D21213D38E
:104AC00011D1D010F03031F133F3F23236F6F7373E
:104AD000F53534F43CFCFD3DFF3F3EFEFA3A3BFB2E
:104AE00039F9F83828E8E929EB2B2AEAEE2E2FEFDE
:104AF0002DEDEC2CE42425E527E7E62622E2E3234E
:104B0000E12120E0A06061A163A3A26266A6A7677D
:104B1000A56564A46CACAD6DAF6F6EAEAA6A6BABED
:104B200069A9A86878B8B979BB7B7ABABE7E7FBF1D
:104B30007DBDBC7CB47475B577B7B67672B2B3730D
:104B4000B17170B0509091519353529296565797BD
:104B5000559594549C5C5D9D5F9F9E5E5A9A9B5BAD
:104B600099595898884849894B8B8A4A4E8E8F4F5D
:104B70008D4D4C8C448485458747468682424383CD
:104B8000418180400000000001020304282065529A
:104B900063765374617465203D3D20535441544500
:104BA0005F52585F494E49542029207C7C202820A0
:104BB000655263765374617465203D3D20535441C2
:104BC00054455F52585F5243562029207C7C202850
:104BD00020655263765374617465203D3D205354C3
:104BE0004154455F52585F4552524F522029002E82
:104BF0002E2F4170702F4D6F646275732F72747514
:104C00002F6D627274752E6300282065526376538F
:104C100074617465203D3D2053544154455F5258A2
:104C20005F5243562029207C7C20282065526376E1
:104C30005374617465203D3D2053544154455F5287
:104C4000585F574149545F454F462029002E2E2F6B
:104C50004170702F4D6F646275732F617363696962
:104C60002F6D6261736369692E6300008C4C0008CC
:104C7000000000209800000010010008244D0008EA
:104C800098000020881C00002C010008030100008F
:104C900001000001000001000001000000A24A0420
:104CA000020000001100000045250008040000007B
:104CB0004524000803000000ED2300081000000058
:104CC0003526000806000000A9250008170000008E
:104CD000A7240008010000000923000805000000C7
:104CE000652500080F000000DB2500080200000019
:104CF0007923000800000000000000000000000010
:104D000000000000000000000000000000000000A3
:104D10000000000000000000000000000000000093
:044D2000000000008F
:04000005080001A945
:00000001FF
